:0400000043EF27F0B3
:1000080000C016F001C015F0E1CF17F0E2CF18F0EC
:100018009DAA5ED09EAA5CD0ABA20FD0AB98AECF03
:10002800D7F0AB88010E01014225006E000E432176
:10003800016E00C042F101C043F1ABA40FD0010131
:10004800AB9EAB8E010E4225006E000E4321016E61
:1000580000C042F101C043F1AECFD7F0AECFD7F028
:100068000001D7510D0A19E1010E0101406F000E80
:10007800416F8D0E0001CD25E16E000ECE21E26E9E
:10008800E1CFE1FFE2CFE2FFE66ACDC044F1CEC0A6
:1000980045F1CD6BCE6BD76B1AD08D0ECD25E16EA9
:1000A800000ECE21E26EE1CFE1FFE2CFE2FFD7C042
:1000B800E6FFCDC044F1CEC045F1010ECD25006E5E
:1000C800000ECE21016E00C0CDF001C0CEF09E9A88
:1000D8009DA01FD09EA01DD0010E01013C25006EE1
:1000E800000E3D21016E00C03CF101C03DF1000E43
:1000F8003D5D02E1080E3C5D07E33C6B3D6B010E84
:100108003E6F000E3F6F9D900B0ECF6EDB0ECE6ED6
:100118009E9016C000F015C001F017C0E1FF18C08E
:04012800E2FF1100E1
:0E012C00026A016A006A086A036A000E120085
:0E013A00ACB202D00000FCD790C1ADFF1200A5
:0C01480072B201D0FDD790C173FF12000D
:100154000B840BAEB5EF00F0010E036E026A016A68
:0A016400006A0A360232FF0E120094
:08016E000AAE029E000E120011
:100176000B820BAEC5EF00F00368026801680068E9
:080186000A360232FF0E1200DE
:10018E00F250026EF29E0500FF6A0150FE6E0050A4
:08019E00FD6E02BEF28E12009C
:1001A600C7B409D01F0EC514016E0150000A03E141
:0A01B600010E006E01D0006A120075
:1001C0000CB022EF01F00CA2C8EF01F00E6A000E95
:1001D000026439EF01F0F00E0214D8A404EF01F02C
:1001E000023A01380F0B02260138F00B016E00387D
:1001F0000F0B01260038F00B006E08380F0B00269D
:100200000838F00B086E0E84D89002BE1DEF01F086
:1002100008360036013602360E2A02BE1DEF01F006
:1002200008360036013602360E2A02BE1DEF01F0F6
:1002300008360036013602360E2A0E500364BEEF31
:1002400001F0035E0BBC08AEC3EF01F0D880800E56
:1002500008640030000E002201220222D8A0C3EF61
:1002600001F0023201320032034AC8EF01F0C3EF5D
:1002700001F001C002F000C001F008C000F0086AFF
:10028000000E0E86026470EF01F0F00E0214D8A486
:1002900058EF01F0023A01380F0B02260138F00B3B
:1002A000016E00380F0B01260038F00B006E0E8433
:1002B000D89002BE1DEF01F00036013602360E2A3C
:1002C00002BE1DEF01F00036013602360E2A02BED4
:1002D0001DEF01F00036013602360E2A1DEF01F047
:1002E00001C002F000C001F0006A000E0E960E88F8
:1002F00002649DEF01F0F00E0214D8A488EF01F023
:10030000023A01380F0B02260138F00B016E0E8401
:10031000D89002BE1DEF01F0013602360E2A02BE51
:100320001DEF01F0013602360E2A02BE1DEF01F06C
:10033000013602360E2A1DEF01F001C002F0016AFB
:10034000000E0E860264CDEF01F0F00E0214D8A468
:10035000ACEF01F0023A0E84D89002BE1DEF01F01E
:1003600002360E2A02BE1DEF01F002360E2A02BE30
:100370001DEF01F002360E2A1DEF01F0010E0C6E8A
:10038000E9DED0EF01F0020E0C6EF1DED0EF01F0ED
:10039000040E0C6EF0DED0EF01F0080E0C6EC6DE1F
:0203A000120049
:1003A20019C08AF11AC08BF11BC08CF11CC08DF1EF
:1003B2006B826BA21FD019501A101B101C1019E06F
:1003C20001018A518B118C118D110CE158C0E1FF92
:1003D20059C0E2FF060EE66E56C000F057C001F0AB
:1003E200D5DE08D0010E01018A5F000E8B5B8C5BAB
:0603F2008D5BDFD7120055
:0403F800C5841200A6
:0803FC000B6A0B86FF0E1200D4
:040404006B841200F3
:10040800086A096A000E0762036489EF02F0025065
:1004180006180A6E075003267E0ED8A01AEF02F0BF
:10042800035ED8B08DEF02F01EEF02F0035ED8A095
:1004380091EF02F0028E068E02C00EF001C00BF0A2
:1004480000C00DF000500402F4CF0CF0015005027A
:10045800F4CF00F0F3CF08F00402F3500C26F45068
:100468000822000E00220D500502F3500C26F4500D
:100478000822000E002202500402F3500826F4500D
:10048800002202500502016A000E0122F3500026E4
:10049800F45001220D500602F3500826F4500022B1
:1004A800026A000E012202220B500602F3500026B7
:1004B800F4500122000E02220E500602F3500126CB
:1004C800F450022202BE71EF02F0083600360136FF
:1004D80002360306D8B491EF02F084EF02F0D88018
:1004E800800E08640030000E002201220222D8A0EB
:1004F80084EF02F0023201320032034A8DEF02F03B
:100508000AAE029E000E93EF02F0010E0BDE93EF8F
:1005180002F0020E2CDE93EF02F0040E17DE12003A
:10052800086A080E0C6E003408360450085ED8B00D
:0E05380002D00826D89000360C2EF5D71200FF
:100546000B800BAEAFEF02F0026A0AAEFF0E026E30
:0C055600016E006E0A360232FF0E120029
:100562000D6A086A0050D8B4000C04180A6E0ABE5C
:100572000D1E0B6A04AE02D0041E042A00AE02D085
:10058200001E002A005004100A6E0ABE1FD004503A
:10059200085E003600340836045008260036060E7F
:1005A2000C6E00340836045000B0085E00A0082625
:1005B20000360C2EF6D700A008260BB015D00DAED3
:1005C200000C001E002A081E082A000C04AE09D0E6
:1005D20000BE04D00050086E006AF1D7006A002AFB
:1005E200000C001E0B2AD3D7082A0450085CD8A49A
:0E05F200E6D7086A002A00AEE2D7FF0C12001E
:100600001DC08AF11EC08BF11FC08CF120C08DF17E
:10061000C582C5A21FD01D501E101F10201019E04A
:1006200001018A518B118C118D110CE11AC1E1FF6E
:100630001BC1E2FF060EE66E18C100F019C101F001
:10064000A6DD08D0010E01018A5F000E8B5B8C5B7A
:060650008D5BDFD71200F4
:10065600025006180E6E086A096A0B6A0350076490
:100666001EEF04F006500A6E068E028E03500B6EC5
:100676000750036E000E0B646EEF03F00B50075E1F
:10068600D8B40FEF04F0070E0764DDEF03F0075E42
:1006960000C008F001C000F002C001F0026A074E77
:1006A6000FEF04F00764B2EF03F0075E00C008F036
:1006B60001C000F0016A074E0FEF04F0076490EFE7
:1006C60003F0075E00C008F0006A074E0FEF04F063
:1006D600076477EF03F00AC002F005C001F004C01A
:1006E60000F0086A3BEF05F0030E076482EF03F0A3
:1006F600075E08380F0B086E074E0FEF04F0D89010
:100706000832074E0FEF04F0D8900832074E0FEF6D
:1007160004F0D89008320FEF04F0030E0764A1EF3F
:1007260003F0075E08380F0B086E0038F00B08263A
:1007360000380F0B006E074E0FEF04F0D890003212
:100746000832074E0FEF04F0D89000320832074EF9
:100756000FEF04F0D890003208320FEF04F0030ECA
:100766000764C9EF03F0075E08380F0B086E003800
:10077600F00B082600380F0B006E0138F00B002630
:1007860001380F0B016E074E0FEF04F0D8900132BF
:1007960000320832074E0FEF04F0D89001320032D3
:1007A6000832074E0FEF04F0D890013200320832BB
:1007B6000FEF04F0030E0764FAEF03F0075E083844
:1007C6000F0B086E0038F00B082600380F0B006E72
:1007D6000138F00B002601380F0B016E0238F00BC2
:1007E600012602380F0B026E074E0FEF04F0D89069
:1007F6000232013200320832074E0FEF04F0D89071
:100806000232013200320832074E0FEF04F0D89060
:100816000232013200320832096A000E0EAE03EFD0
:1008260005F0081E001E011E021E082A00220122D3
:10083600022203EF05F00750D8A424EF04F03BEFA3
:1008460005F0096A02C00AF0028E068E0750035CA4
:10085600076ED8B4F6EF04F0070E0764C4EF04F091
:10086600075E0450096E0550046E0650056E066A52
:10087600074EF6EF04F0070E076499EF04F0075EE3
:100886000450096E0550046E056A074EF6EF04F033
:10089600070E076477EF04F0075E0450096E046ADA
:1008A600074EF6EF04F0070E07645EEF04F00AC089
:1008B60002F03BEF05F0030E076469EF04F0075EF4
:1008C60009380F0B096E074EF6EF04F0D89009327F
:1008D600074EF6EF04F0D8900932074EF6EF04F013
:1008E600D8900932F6EF04F0030E076488EF04F09F
:1008F600075E09380F0B096E0438F00B0926043819
:100906000F0B046E074EF6EF04F0D890043209324E
:10091600074EF6EF04F0D89004320932074EF6EF90
:1009260004F0D89004320932F6EF04F0030E07649F
:10093600B0EF04F0075E09380F0B096E0438F00BB0
:10094600092604380F0B046E0538F00B042605380B
:100956000F0B056E074EF6EF04F0D8900532043201
:100966000932074EF6EF04F0D89005320432093208
:10097600074EF6EF04F0D890053204320932F6EF4E
:1009860004F0030E0764E1EF04F0075E09380F0B6D
:10099600096E0438F00B092604380F0B046E05386F
:1009A600F00B042605380F0B056E0638F00B0526EE
:1009B60006380F0B066E074EF6EF04F0D890063297
:1009C600053204320932074EF6EF04F0D8900632AB
:1009D600053204320932074EF6EF04F0D89006329B
:1009E600053204320932086A000E0EAE03EF05F036
:1009F600091E041E051E061E092A042205220622B9
:100A060009500826045000220550012206500222F1
:100A16000EBE1AEF05F0D8A029EF05F0023201321A
:100A260000320832033E29EF05F035EF05F0D8B065
:100A36002FEF05F0000E081E001E011E021E082ADA
:100A46000022012202220A7E2FEF05F0010E0C6E13
:100A5600E0EC00F03DEF05F0020E0C6EE0EC00F06D
:100A66003DEF05F0040E0C6EBBEC00F03DEF05F01B
:060A7600000E0C6E1200E0
:100A7C001DC08CF11EC08DF11FC08EF120C08FF1F6
:100A8C0001018A6B8B6B8B51120802E18A518E0823
:100A9C0009E3D3EC00F0005201E004D001018A4BD1
:100AAC008B2BF1D70101120E8B5D02E18F0E8A5D4B
:100ABC0003E37B0E006E25D0C580C5A021D01D5050
:100ACC001E101F1020101BE08C518D118E118F11D8
:100ADC000FE11AC1E1FF1BC1E2FF050EE66E18C162
:100AEC0000F019C101F0C7EC00F0010E006E09D046
:100AFC00010E01018C5F000E8D5B8E5B8F5BDDD771
:040B0C00006A120069
:100B10009E968AC1C9FF1DC08BF11EC08CF11FC0FB
:100B20008DF120C08EF1C7A422D01D501E101F10C1
:100B300020101CE001018B518C118D118E110FE1E1
:100B40001AC1E1FF1BC1E2FF040EE66E18C100F0FE
:100B500019C101F0C7EC00F0010E006E3BD0010E90
:100B600001018B5F000E8C5B8D5B8E5BDCD71DC043
:100B70008BF11EC08CF11FC08DF120C08EF19EB68E
:100B800022D01D501E101F1020101CE001018B519F
:100B90008C118D118E110FE11AC1E1FF1BC1E2FF13
:100BA000040EE66E18C100F019C101F0C7EC00F0A8
:100BB000010E006E0FD0010E01018B5F000E8C5BE9
:100BC0008D5B8E5BDCD7C5BC02D0006A03D0C584C8
:060BD000020E006E12008F
:100BD6000134083609360450085E0550D8A0053C95
:100BE600095E003601360F0E0C6E013408360936E2
:100BF600045000A006D0085E0550D8A0053C095E4A
:100C060005D008260550D8B0053C09260036013621
:100C16000C2EEBD700B006D0045008260550D8B0ED
:080C2600053C09260000120044
:100C2E000B6A0C6A086A0350D8B49BEF06F002C038
:100C3E000AF0028E9E0E035E03AE8BEF06F0036C7F
:100C4E00080E035CD8A058EF06F0036E083600C0FD
:100C5E0008F001C000F002C001F0026A080E035C49
:100C6E00D8A058EF06F0036E083600C008F001C099
:100C7E0000F0016A080E035CD8A058EF06F0036E70
:100C8E00083600C008F0006A080E035CD8A058EFC2
:100C9E0006F0036E0836086A0350D8A4D89064EFA5
:100CAE0006F00350D8B464EF06F0D8900232013249
:100CBE0000320832032E5CEF06F00BBC08A075EF75
:100CCE0006F0D8A075EF06F0082AD8B4002AD8B4DA
:100CDE00012AD8B4022A02BE9FEF06F00AAE9BEF9D
:100CEE0006F0021E011E001E081E082AD8B4002A95
:100CFE00D8B4012AD8B4022A9BEF06F0026A016A20
:100D0E00006A086A9BEF06F00B800BAEA5EF06F0AB
:100D1E00026A0AAEA5EF06F0026E016E006E086E54
:100D2E000A360232A5EF06F00C6A000EA6EF06F0A8
:100D3E00010E0C6E000E00DCA6EF06F0FF0E025048
:100D4E00036E0150026E0050016E0850006E1200CC
:100D5E0001018551390806E3300E855D03E3010E6E
:080D6E00006E01D0006A1200C2
:100D76006E0E0101855DD8A0CAD0640E046E85C1D1
:100D860000F094EC02F0120E0024056E066A000EC6
:100D9600062205C000F006C001F0000E06BEFF0EDA
:100DA600026E036E003600900136023603360036B8
:100DB6000090013602360336CB0E0024F66E550E31
:100DC6000120F76E000E0220F86E0900F5CF00F044
:100DD6000900F5CF01F00900F5CF02F00900F5CFC3
:100DE60003F0000E046E000E056E000E066E7E0EFB
:100DF600076E04EC02F000C086F101C087F102C064
:100E060088F103C089F1640E046E85C100F094EC8C
:100E160002F008C000F00A0E046E94EC02F0090E0F
:100E26000024056E066A000E062205C000F006C004
:100E360001F0000E06BEFF0E026E036E0036009035
:100E46000136023603360036009001360236033686
:100E5600CB0E0024F66E550E0120F76E000E022012
:100E6600F86E0900F5CF00F00900F5CF01F0090092
:100E7600F5CF02F00900F5CF03F086C104F087C173
:100E860005F088C106F089C107F004EC02F000C045
:100E960086F101C087F102C088F103C089F10A0E0C
:100EA600046E85C100F094EC02F008C000F000C0AA
:100EB60001F0000E026E036E046E013601900236DA
:100EC6000336043601360190023603360436CB0E5D
:100ED6000124F66E550E0220F76E000E0320F86E02
:100EE6000900F5CF00F00900F5CF01F00900F5CFB4
:100EF60002F00900F5CF03F086C104F087C105F0C2
:100F060088C106F089C107F004EC02F0B1D0855122
:100F16000A08D8B07ED00A0E046E85C100F094ECA3
:100F260002F0090E0024056E066A000E062205C0B0
:100F360000F006C001F0000E06BEFF0E026E036E44
:100F46000036009001360236033600360090013630
:100F560002360336CB0E0024F66E550E0120F76ED0
:100F6600000E0220F86E0900F5CF00F00900F5CF5B
:100F760001F00900F5CF02F00900F5CF03F0000EED
:100F8600046E000E056E000E066E7E0E076E04ECF5
:100F960002F000C086F101C087F102C088F103C0EB
:100FA60089F10A0E046E85C100F094EC02F008C0C7
:100FB60000F000C001F0000E026E036E046E0136F2
:100FC60001900236033604360136019002360336A6
:100FD6000436CB0E0124F66E550E0220F76E000E77
:100FE6000320F86E0900F5CF00F00900F5CF01F0F7
:100FF6000900F5CF02F00900F5CF03F086C104F031
:1010060087C105F088C106F089C107F004EC02F03B
:101016002FD085C100F0000E016E026E036E003601
:10102600009001360236033600360090013602364D
:101036000336CB0E0024F66E550E0120F76E000E19
:101046000220F86E0900F5CF00F00900F5CF01F097
:101056000900F5CF02F00900F5CF03F0000E046E8B
:10106600000E056E000E066E7E0E076E04EC02F094
:02107600120066
:1010780003500718D8A450EF08F002500618D8A457
:1010880050EF08F001500518D8A450EF08F00050B0
:0E1098000418D8B4D8841200D89412001200A4
:1010A6000A6A0350D8A40A800750D8A40A820A50B4
:1010B600D8B4B6EF08F0030AD8B46FEF08F00AB058
:1010C6006AEF08F006AEB4EF08F0B2EF08F002AE31
:1010D600B2EF08F0B4EF08F00250800B0A6E029EE1
:1010E6000650800B069E0A18D8B480EF08F00A5006
:1010F600D8B4B2EF08F0B4EF08F00750035CD8B4E8
:101106008AEF08F0D8A0A6EF08F0ACEF08F006507A
:10111600025CD8B494EF08F0D8A0A6EF08F0ACEFC4
:1011260008F00550015CD8B49EEF08F0D8A0A6EFF1
:1011360008F0ACEF08F00450005CD8B4B6EF08F045
:10114600D8B0ACEF08F00A52D8B4B4EF08F0B2EF5A
:1011560008F00A52D8B4B2EF08F0B4EF08F0D8801D
:0E1166001200D8901200D880D8841200120017
:10117400800E01018519006E800E000A005CD8B053
:101184006DD185510008016E01C085F1800E0118F2
:10119400006E800E6E0A005CD8A0C0D0640E046E8F
:1011A40085C100F0B1EC02F0120E0024056E000EB1
:1011B40000BEFF0E066E000E062205C000F006C03B
:1011C40001F0000E06BEFF0E026E036E00360090A4
:1011D40001360236033600360090013602360336F5
:1011E400CB0E0024F66E550E0120F76E000E022081
:1011F400F86E0900F5CF86F10900F5CF87F10900F3
:10120400F5CF88F10900F5CF89F1640E046E85C12C
:1012140000F0B1EC02F008C000F00A0E046EB1EC6C
:1012240002F0090E0024056E000E00BEFF0E066ECD
:10123400000E062205C000F006C001F0000E06BE36
:10124400FF0E026E036E003600900136023603363E
:1012540000360090013602360336CB0E0024F66EBB
:10126400550E0120F76E000E0220F86E0900F5CF2E
:1012740000F00900F5CF01F00900F5CF02F00900F4
:10128400F5CF03F086C104F087C105F088C106F0EC
:1012940089C107F004EC02F000C086F101C087F1B7
:1012A40002C088F103C089F10A0E046E85C100F002
:1012B400B1EC02F008C000F000C001F0000E00BE66
:1012C400FF0E026E036E046E013601900236033681
:1012D400043601360190023603360436CB0E01245F
:1012E400F66E550E0220F76E000E0320F86E09000C
:1012F400F5CF00F00900F5CF01F00900F5CF02F0B9
:101304000900F5CF03F086C104F087C105F088C158
:1013140006F089C107F004EC02F007D2800E0A0A35
:10132400006E800E8519005C71E20A0E046E85C1A0
:1013340000F0B1EC02F0090E0024056E000E00BEB0
:10134400FF0E066E000E062205C000F006C001F076
:10135400000E06BEFF0E026E036E003600900136CC
:101364000236033600360090013602360336CB0EC1
:101374000024F66E550E0120F76E000E0220F86E62
:101384000900F5CF86F10900F5CF87F10900F5CF03
:1013940088F10900F5CF89F10A0E046E85C100F0C9
:1013A400B1EC02F008C000F000C001F0000E00BE75
:1013B400FF0E026E036E046E013601900236033690
:1013C400043601360190023603360436CB0E01246E
:1013D400F66E550E0220F76E000E0320F86E09001B
:1013E400F5CF00F00900F5CF01F00900F5CF02F0C8
:1013F4000900F5CF03F086C104F087C105F088C168
:1014040006F089C107F004EC02F08FD185C100F029
:10141400000E85BFFF0E016E026E036E0036009053
:1014240001360236033600360090013602360336A2
:10143400CB0E0024F66E550E0120F76E000E02202E
:10144400F86E0900F5CF00F00900F5CF01F00900AE
:10145400F5CF02F00900F5CF03F067D1800E8519AE
:10146400006E800E6E0A005CD8A0C0D0640E046EBC
:1014740085C100F0B1EC02F0120E0024056E000EDE
:1014840000BEFF0E066E000E062205C000F006C068
:1014940001F0000E06BEFF0E026E036E00360090D1
:1014A4000136023603360036009001360236033622
:1014B400FF0E0024F66E550E0120F76E000E02207A
:1014C400F86E0900F5CF86F10900F5CF87F1090020
:1014D400F5CF88F10900F5CF89F1640E046E85C15A
:1014E40000F0B1EC02F008C000F00A0E046EB1EC9A
:1014F40002F0090E0024056E000E00BEFF0E066EFB
:10150400000E062205C000F006C001F0000E06BE63
:10151400FF0E026E036E003600900136023603366B
:1015240000360090013602360336FF0E0024F66EB4
:10153400550E0120F76E000E0220F86E0900F5CF5B
:1015440000F00900F5CF01F00900F5CF02F0090021
:10155400F5CF03F086C104F087C105F088C106F019
:1015640089C107F004EC02F000C086F101C087F1E4
:1015740002C088F103C089F10A0E046E85C100F02F
:10158400B1EC02F008C000F000C001F0000E00BE93
:10159400FF0E026E036E046E0136019002360336AE
:1015A400043601360190023603360436FF0E012458
:1015B400F66E550E0220F76E000E0320F86E090039
:1015C400F5CF00F00900F5CF01F00900F5CF02F0E6
:1015D4000900F5CF03F086C104F087C105F088C186
:1015E40006F089C107F004EC02F09FD0800E0A0ACD
:1015F400006E800E8519005C71E20A0E046E85C1CE
:1016040000F0B1EC02F0090E0024056E000E00BEDD
:10161400FF0E066E000E062205C000F006C001F0A3
:10162400000E06BEFF0E026E036E003600900136F9
:101634000236033600360090013602360336FF0EBA
:101644000024F66E550E0120F76E000E0220F86E8F
:101654000900F5CF86F10900F5CF87F10900F5CF30
:1016640088F10900F5CF89F10A0E046E85C100F0F6
:10167400B1EC02F008C000F000C001F0000E00BEA2
:10168400FF0E026E036E046E0136019002360336BD
:10169400043601360190023603360436FF0E012467
:1016A400F66E550E0220F76E000E0320F86E090048
:1016B400F5CF00F00900F5CF01F00900F5CF02F0F5
:1016C4000900F5CF03F086C104F087C105F088C195
:1016D40006F089C107F004EC02F027D085C100F0C0
:1016E400000E85BFFF0E016E026E036E0036009081
:1016F40001360236033600360090013602360336D0
:10170400FF0E0024F66E550E0120F76E000E022027
:10171400F86E0900F5CF00F00900F5CF01F00900DB
:0C172400F5CF02F00900F5CF03F0120031
:101730000050086E0150006E0250016E0350026EA0
:10174000036A0B6A0C6A9E0E036E0A6A020E0C6E26
:06175000E0EC00F01200C5
:101756000C6A0E6A0250D8A4C4EF0BF001C002F066
:1017660000C001F0006A0E860250D8A4C4EF0BF048
:1017760001C002F0016A0E960E880250D8B4D6EF68
:101786000BF00E50035ED8A4D8A0DCEF0BF0D89077
:1017960002BEE2EF0BF0003601360236032ECBEF27
:1017A6000BF0DCEF0BF0010E0C6E96EC00F0E6EFA2
:1017B6000BF0020E0C6EAAEC00F0E6EF0BF0040E36
:0817C6000C6EB7EC00F01200FC
:0817CE00067E2BEC03F0120073
:1017D6000B6A0A6A096A086A0E6A033408360450F4
:1017E600085E0550D8A0053C095E0650D8A0063C08
:1017F6000A5E0750D8A0073C0B5EE86AD8A0010E27
:101806000E5E0336070E0C6E0334083609360A36AA
:101816000B360E36045003A012D0085E0550D8A031
:10182600053C095E0650D8A0063C0A5E0750D8A0C3
:10183600073C0B5EE86AD8A0010E0E5E11D00826A2
:101846000550D8B0053C09260650D8B0063C0A26F5
:101856000750D8B0073C0B26E86AD8B0010E0E2612
:1018660003360C2ED1D70234083609360A360B3623
:101876000E36045003A012D0085E0550D8A0053CD1
:10188600095E0650D8A0063C0A5E0750D8A0073C61
:101896000B5EE86AD8A0010E0E5E11D00826055030
:1018A600D8B0053C09260650D8B0063C0A26075093
:1018B600D8B0073C0B26E86AD8B0010E0E260236D1
:1018C600070E0C6E0234083609360A360B360E360B
:1018D600045002A012D0085E0550D8A0053C095E4F
:1018E6000650D8A0063C0A5E0750D8A0073C0B5EFF
:1018F600E86AD8A0010E0E5E11D008260550D8B0B1
:10190600053C09260650D8B0063C0A260750D8B032
:10191600073C0B26E86AD8B0010E0E2602360C2EBE
:10192600D1D70134083609360A360B360E3604503E
:1019360002A012D0085E0550D8A0053C095E0650EC
:10194600D8A0063C0A5E0750D8A0073C0B5EE86AA2
:10195600D8A0010E0E5E11D008260550D8B0053C61
:1019660009260650D8B0063C0A260750D8B0073CD0
:101976000B26E86AD8B0010E0E260136070E0C6E4D
:101986000134083609360A360B360E36045001A0E5
:1019960012D0085E0550D8A0053C095E0650D8A0B6
:1019A600063C0A5E0750D8A0073C0B5EE86AD8A042
:1019B600010E0E5E11D008260550D8B0053C09264A
:1019C6000650D8B0063C0A260750D8B0073C0B266E
:1019D600E86AD8B0010E0E2601360C2ED1D7003497
:1019E600083609360A360B360E36045001A012D0D8
:1019F600085E0550D8A0053C095E0650D8A0063CF6
:101A06000A5E0750D8A0073C0B5EE86AD8A0010E14
:101A16000E5E11D008260550D8B0053C09260650A2
:101A2600D8B0063C0A260750D8B0073C0B26E86A11
:101A3600D8B0010E0E260036070E0C6E003408369E
:101A460009360A360B360E36045000A012D0085E50
:101A56000550D8A0053C095E0650D8A0063C0A5E93
:101A66000750D8A0073C0B5EE86AD8A0010E0E5EB0
:101A760011D008260550D8B0053C09260650D8B026
:101A8600063C0A260750D8B0073C0B26E86AD8B0B1
:101A9600010E0E2600360C2ED1D700B00ED0045003
:101AA60008260550D8B0053C09260650D8B0063C95
:0C1AB6000A260750D8B0073C0B2612008F
:101AC2000450000A08E10550000A05E1FF0E006E0D
:101AD2007F0E016E58D00D6A096A086A0150001023
:101AE200D8B4000C015005180A6E0ABE0D1E0B6A0E
:101AF20005AE05D0041E051E042AD8B4052A01AE7F
:101B020005D0001E011E002AD8B4012A015005107A
:101B12000A6E0ABE10D0EBEC05F00BB020D00DAE71
:101B2200000C001E011E002AD8B4012A081E091E3C
:101B3200082AD8B4092A000C05AE0DD001BE07D080
:101B42000150096E0050086E016A006AE8D7016A06
:101B5200006A002A000C011E001E0B2ADDD7082A8B
:101B6200D8B4092A0450085CD8A4D9D70550095C16
:101B7200D8A4D5D7096A086A002AD8B4012A01AEC6
:081B8200CED70000FF0C120099
:101B8A003EEC05F085C18AF188EC05F000C087F1CA
:101B9A00000E016EFF0E011802E1FF0E0018D8B404
:101BAA00C69E86C18AF188EC05F000C087F1FCEC7C
:081BBA0001F087C100F01200E8
:101BC2000B6A0C6A0A6A086A0350D8B469EF0EF00D
:101BD200028E9E0E035E03BEF4EF0DF0D8B4F4EF56
:101BE2000DF059EF0EF0036C080E035CD8A026EF3F
:101BF2000EF0036E083600C008F001C000F002C00B
:101C020001F0026A080E035CD8A026EF0EF0036E04
:101C1200083600C008F001C000F0016A080E035C3B
:101C2200D8A026EF0EF0036E083600C008F0006A56
:101C3200080E035CD8A026EF0EF0036E0836086A81
:101C42000350D8A4D89032EF0EF00350D8B432EF3C
:101C52000EF0D8900232013200320832032E2AEFFF
:101C62000EF00BBC08A043EF0EF0D8A043EF0EF02D
:101C7200082AD8B4002AD8B4012AD8B4022A02BE4B
:101C82006DEF0EF00AAE69EF0EF0021E011E001E8D
:101C9200081E082AD8B4002AD8B4012AD8B4022AC5
:101CA20069EF0EF0026A016A006A086A69EF0EF0D3
:101CB2000B800BAE73EF0EF0026A0AAE73EF0EF0FA
:101CC200026E016E006E086E0A36023273EF0EF07B
:101CD200000E0C6A74EF0EF0010E0C6EA3EC02F013
:101CE20074EF0EF0FF0E0250036E0150026E0050B0
:081CF200016E0850006E1200A3
:101CFA000B6A0A6A096A00500402F4CF09F0F3CFAA
:101D0A0008F001500502F4CF0BF0F3CF0AF00050AF
:101D1A000502F3500926F4500A22E86A0B22015000
:101D2A000402F3500926F4500A22E86A0B2208C07A
:101D3A0000F009C001F00AC002F00BC003F0120063
:101D4A000450000A12E10550000A0FE10650000A89
:101D5A000CE10750000A09E1FF0E006EFF0E016E4A
:101D6A007F0E026EFF0E036EA8D0086A096A07503A
:101D7A00D8B450EF0FF00350D8B455EF0FF002501B
:101D8A0006180A6E028E068E0E6A02C008F001C09C
:101D9A000CF000C00DF004500D5E0550D8A0053CB3
:101DAA000C5E0650D8A0063C085E086A0C6A0D6AEA
:101DBA00D8A0E7EF0EF0D890023201320032083292
:101DCA00010E0E6E0750035ED8A0F4EF0EF07E0EE1
:101DDA000E240326D8B05AEF0FF0FAEF0EF07E0E5B
:101DEA000E240326D8A05FEF0FF0180E0B6E0D36E7
:101DFA000C3608360036013602360E360450005EBE
:101E0A000550D8A0053C015E0650D8A0063C025EEB
:101E1A0006340E120EA015EF0FF00D8020EF0FF012
:101E2A00045000260550D8B0053C01260650D8B00B
:101E3A00062802260D900B2EFCEF0EF046EF0FF04F
:101E4A00D8900036013602360E360450005E055030
:101E5A00D8A0053C015E0650D8A0063C025E0634B6
:101E6A000E10010B0D26D8B00C2AD8B4082AD8A413
:101E7A0046EF0FF008320C320D32032AD8B45AEF6B
:101E8A000FF00AAE089E0850026E0C50016E0D50FB
:101E9A00006E62EF0FF0010EFEEC01F062EF0FF040
:101EAA00020E96EC00F062EF0FF0040EBBEC00F0AD
:0C1EBA0062EF0FF0080EAAEC00F012001E
:101EC6000B6A0350D8B4A9EF0FF002500A6E028EC7
:101ED6008E0E035E03AEADEF0FF0036C080E035CCF
:101EE600D8A088EF0FF0036E013602C001F0026A37
:101EF600080E035CD8A088EF0FF0036E0136016A66
:101F06000350D8A4D89092EF0FF00350D8B492EFB4
:101F16000FF0D89002320132032E8CEF0FF00BBC7B
:101F260001A09FEF0FF0D8A09FEF0FF0012AD8B4C1
:101F3600022A02BEBCEF0FF00AAEC2EF0FF0021E7D
:101F4600011E012AD8B4022AC2EF0FF0026A016A02
:101F5600C2EF0FF00B800BAEC6EF0FF0026A0AAEAF
:101F6600C6EF0FF0FF0E026E016E0A360232C6EFA2
:101F76000FF0010E0C6EA3EC02F0C8EF0FF0000E8E
:101F86000C6EC8EF0FF0FF0E0C6E0150006E025083
:041F9600016E1200C6
:101F9A0000C008F00150006E016A026A036A0B6A07
:101FAA000C6A016A026A036A960E036E0A6A00AE36
:101FBA00E5EF0FF0081E001E082AD8B4002A0A8E80
:101FCA0000C001F008C000F0086A026AABEC0BF02E
:021FDA001200F3
:101FDC005DC1F6FF5EC1F7FF5FC1F8FF0900F5CFE9
:101FEC0000F0005212E05DC1F6FF5EC1F7FF5FC169
:101FFC00F8FF0900F5CF90F19DEC00F0010E010106
:0C200C005D27000E5E235F23E3D7120067
:0A201800750E0D6E0D2EFED712009E
:1020220001017D6B7E6B716B726B5FC100F060C1F1
:1020320001F061C102F0010E5F27000E60236123EF
:1020420000C0F6FF01C0F7FF02C0F8FF0900F5CF9C
:1020520000F000C06EF10052D8B41DEF20F06E51B6
:10206200250A0BE05DC1E1FF5EC1E2FF6EC1E6FF42
:102072005D4B5E2B7D4B7E2BD8D76F6B706B716B7C
:10208200726B23D07187010E5F27000E60236123DC
:1020920059D07181010E5F27000E6023612352D057
:1020A2007183010E5F27000E602361234BD072877C
:1020B200010E5F27000E6023612344D07185010E5B
:1020C2005F27000E602361233DD05FC1F6FF60C130
:1020D200F7FF61C1F8FF0900F5CF01F001502D0AA9
:1020E200D1E05FC1F6FF60C1F7FF61C1F8FF0900EF
:1020F200F5CF01F00150200ACCE05FC1F6FF60C1CC
:10210200F7FF61C1F8FF0900F5CF01F001502B0A7A
:10211200C7E05FC1F6FF60C1F7FF61C1F8FF0900C8
:10212200F5CF01F00150230AC2E05FC1F6FF60C1A2
:10213200F7FF61C1F8FF0900F5CF01F00150300A45
:10214200BDE001D09ED771A301D0719171A701D0DA
:1021520071955FC1F6FF60C1F7FF61C1F8FF090029
:10216200F5CF00F0000E016E00C085F1AFEC06F075
:10217200005235E06F6B706B6FC100F070C101F0FF
:102182000A0E046E000E056EB7DD5FC1F6FF60C178
:10219200F7FF61C1F8FF0900F5CF02F002500024F9
:1021A2006F6F000E0120706F300E6F5F000E705B5C
:1021B200010E5F27000E602361235FC1F6FF60C13D
:1021C200F7FF61C1F8FF0900F5CF00F0000E016EC4
:1021D20000C085F1AFEC06F00052CEE133D05FC112
:1021E200F6FF60C1F7FF61C1F8FF0900F5CF01F00A
:1021F20001502A0A27E162C1E9FF63C1EAFFEECF7B
:1022020000F0EECF01F000C0E9FF01C0EAFFEECF1F
:102212006FF1EECF70F162C1E9FF63C1EAFF020E16
:10222200EE24006E000EEE20016E62C1E1FF63C17A
:10223200E2FF00C0E6FF01C0E6FF010E5F27000ECD
:10224200602361235FC1F6FF60C1F7FF61C1F8FF40
:102252000900F5CF01F001502E0A6FE1010E5F2750
:10226200000E602361235FC1F6FF60C1F7FF61C109
:10227200F8FF0900F5CF01F001502A0A28E162C1F6
:10228200E9FF63C1EAFFEECF00F0EECF01F000C03C
:10229200E9FF01C0EAFFEECF6CF1EECF6DF162C152
:1022A200E9FF63C1EAFF020EEE24006E000EEE208B
:1022B200016E62C1E1FF63C1E2FF00C0E6FF01C03F
:1022C200E6FF010E5F27000E6023612335D06C6BA1
:1022D2006D6B5FC1F6FF60C1F7FF61C1F8FF0900D6
:1022E200F5CF00F0000E016E00C085F1AFEC06F0F4
:1022F200005222E06CC100F06DC101F00A0E046EC2
:10230200000E056EF9DC5FC1F6FF60C1F7FF61C127
:10231200F8FF0900F5CF02F0025000246C6F000EA6
:1023220001206D6F300E6C5F000E6D5B010E5F273A
:10233200000E60236123CDD703D06C6B6D6B728965
:102342005FC100F060C101F061C102F0010E5F27C0
:10235200000E6023612300C0F6FF01C0F7FF02C038
:10236200F8FF0900F5CF6EF1F9D07DC100F07EC112
:1023720001F021EF20F07189E3D772852ED1718BA4
:1023820072812BD1728329D1718D27D126D1718B84
:10239200718F23D162C1E9FF63C1EAFFEECF00F082
:1023A200EECF01F000C0E9FF01C0EAFFEECF79F104
:1023B200EECF7AF162C1E9FF63C1EAFF020EEE24B9
:1023C200006E000EEE20016E62C1E1FF63C1E2FF0A
:1023D20000C0E6FF01C0E6FF000E7A1902E1000E1E
:1023E200791904E1210E796F000E7A6F7B6B7C6B99
:1023F2007B517925E96E7C517A21EA6EEE520BE02F
:10240200010E7B25006E000E7C21016E00C07BF167
:1024120001C07CF1EDD76C516D110AE07C516D5D0C
:1024220002E17B516C5D04E26CC17BF16DC17CF118
:1024320070517C5D02E16F517B5D05E27B516F5F04
:102442007C51705B02D06F6B706B71B716D06FC12D
:1024520000F070C101F0010E6F5F000E705B005062
:1024620001100BE05DC1E1FF5EC1E2FF200EE66EEE
:102472005D4B5E2B7D4B7E2BEAD77BC102F07CC18C
:1024820003F0010E7B5D006E000E7C59016E00C0F0
:102492007BF101C07CF10250031019E079C1E9FF20
:1024A2007AC1EAFF5DC1E1FF5EC1E2FFEECFE6FF66
:1024B2005D4B5E2B010E7925006E000E7A21016EB6
:1024C20000C079F101C07AF17D4B7E2BD6D771A77E
:1024D20016D06FC100F070C101F0010E6F5F000EE7
:1024E200705B005001100BE05DC1E1FF5EC1E2FFD5
:1024F200200EE66E5D4B5E2B7D4B7E2BEAD795D58B
:1025020062C1E9FF63C1EAFFEECF00F0EECF01F056
:1025120000C0E9FF01C0EAFFEECF6EF162C1E9FF40
:1025220063C1EAFF020EEE24006E000EEE20016E81
:1025320062C1E1FF63C1E2FF00C0E6FF01C0E6FF46
:102542006E0E796F010E7A6F010E7B6F000E7C6F3B
:1025520062D7C00E7113000E72133FD06E51000A83
:10256200D8B403D76E516C0AD8B405D76E514C0A51
:10257200D8B401D76E51660AD8B4FFD66E51450A57
:10258200D8B4FDD66E51650AD8B4FAD66E51670A30
:10259200D8B4F8D66E516F0AD8B4F6D66E51640A22
:1025A200D8B4F4D66E51690AD8B4F0D66E51700A16
:1025B200D8B4EDD66E51580AD8B4E9D66E51780A1D
:1025C200D8B4E6D66E51730AD8B4E4D66E51630A13
:1025D20097E06E51750ABDE0B3D7000E7115006E1B
:1025E2007251070B016E00500110D8B4C4EF1BF0FA
:1025F20072A904D0060E6C6F000E6D6F62C1E9FF06
:1026020063C1EAFFEECF00F0EECF01F000C0E9FFB8
:1026120001C0EAFFEECF73F1EECF74F1EECF75F1A8
:10262200EECF76F162C1E9FF63C1EAFF040EEE2448
:10263200006E000EEE20016E62C1E1FF63C1E2FF97
:1026420000C0E6FF01C0E6FF046A056A066A076A7F
:1026520073C100F074C101F075C102F076C103F0DC
:1026620053EC08F0010ED8B0000E006E005205E0E7
:10267200757F030E7113000E7213776B786B73C143
:1026820000F074C101F075C102F076C103F0046A72
:10269200056A066A076A3CEC08F0000ED8A4010E2F
:1026A200006E0052D8B48AD076C100F0016A026A84
:1026B200036AFF0E0016000E01167E0E005E000E6B
:1026C200015A00C077F101C078F1010E005E000EE0
:1026D200015A00C077F101C078F1030E046E000EBA
:1026E200056E7DEC0EF000C077F101C078F10A0EA4
:1026F200046E000E056E61EC0DF000C077F101C0B2
:1027020078F1800E0118026E800E025C02E1000E6A
:10271200005C05E2010E0101775F000E785B0101AA
:1027220077510008856FBAEC08F073C104F074C1E8
:1027320005F075C106F076C107F004EC02F000C0A6
:1027420079F101C07AF102C07BF103C07CF1000E85
:10275200046E000E056E000E066E7F0E076E79C1C6
:1027620000F07AC101F07BC102F07CC103F053ECAE
:1027720008F0010ED8B0000E006E005205E0010E06
:10278200775F000E785B1AD0000E046E000E056EA5
:10279200200E066E820E076E79C100F07AC101F03A
:1027A2007BC102F07CC103F053EC08F0000ED8B0FC
:1027B200010E006E005202E0774B782B800E006E05
:1027C200800E7819005C02E17751000803E3010EE4
:1027D2006E6F02D077C16EF172B118D072A315D0AC
:1027E200800E7819006E7F0E005C02E1FC0E775DB0
:1027F2000BE3800E7819006E800E6D19005C02E109
:102802006C51775D01E201D001D0EFD36C516D11B3
:1028120006E072A304D0010E6C5F000E6D5B6D5179
:10282200000802E16C51080803E2080E6E6F02D044
:102832006CC16EF173C100F074C101F075C102F098
:1028420076C103F0046A056A066A076A3CEC08F07E
:10285200000ED8A4010E006E0052D8B44BD177C13D
:1028620085F1BAEC08F000C004F001C005F002C026
:1028720006F003C007F073C100F074C101F075C126
:1028820002F076C103F0A5EC0EF000C073F101C0B6
:1028920074F102C075F103C076F101016E510008B6
:1028A200856FBAEC08F000C004F001C005F002C068
:1028B20006F003C007F073C100F074C101F075C1E6
:1028C20002F076C103F0A5EC0EF000C07FF101C06A
:1028D20080F102C081F103C082F17FC173F180C136
:1028E20074F181C175F182C176F17FC100F080C1BE
:1028F20001F081C102F082C103F0E1EC0DF098EC2D
:102902000BF000C004F001C005F002C006F003C0E5
:1029120007F07FC100F080C101F081C102F082C1E5
:1029220003F0E7EC0BF0000E046E000E056E000ED5
:10293200066E7E0E076E53EC08F0000ED8B0010E44
:10294200006E00521AE073C100F074C101F075C14B
:1029520002F076C103F0000E046E000E056E000E4A
:10296200066E7E0E076E2BEC03F000C073F101C001
:1029720074F102C075F103C076F173C100F074C145
:1029820001F075C102F076C103F0E1EC0DF0010136
:102992006E51010F096E0A6A000E0A2209C004F084
:1029A2000AC005F0000E0ABEFF0E066E076E043660
:1029B2000490053606360736043604900536063688
:1029C2000736970E0424F66E560E0520F76E000E9B
:1029D2000620F86E0900F5CF05F00900F5CF06F0E4
:1029E2000900F5CF07F00900F5CF08F00850035CA5
:1029F20008E10750025C05E10650015C02E1055066
:102A0200005C1EE3010173C100F074C101F075C1E5
:102A120002F076C103F0CD0E046ECC0E056E4C0EA4
:102A2200066E7B0E076E04EC02F000C073F101C06B
:102A320074F102C075F103C076F1774B782B5AD04E
:102A420073C100F074C101F075C102F076C103F0E8
:102A5200E1EC0DF06EC104F0000E056E066E076E1D
:102A620004360490053606360736043604900536D9
:102A720006360736970E0424F66E560E0520F76EBC
:102A8200000E0620F86E0900F5CF05F00900F5CF1B
:102A920006F00900F5CF07F00900F5CF08F008505D
:102AA200035C08E10750025C05E10650015C02E1AB
:102AB2000550005C1FE2010173C100F074C101F016
:102AC20075C102F076C103F0000E046E000E056EB1
:102AD200200E066E820E076E04EC02F000C073F147
:102AE20001C074F102C075F103C076F1010E775F87
:102AF200000E785B010172A393D072B791D0800E61
:102B0200000A006E800E6D19005C02E16C510A0829
:102B120004E20A0E6C6F000E6D6F73C100F074C197
:102B220001F075C102F076C103F0E1EC0DF000C0D6
:102B320079F101C07AF102C07BF103C07CF17951D5
:102B42007A117B117C1142E00A0E046E000E056EB2
:102B5200066E076E79C100F07AC101F07BC102F006
:102B62007CC103F0EBEC0BF008C000F009C001F0EF
:102B72000AC002F00BC003F0000E046E031808E155
:102B82000450021805E10450011802E10050000A45
:102B92001DE1010E6C5F000E6D5B0A0E046E000EED
:102BA200056E066E076E79C100F07AC101F07BC135
:102BB20002F07CC103F0EBEC0BF000C079F101C034
:102BC2007AF102C07BF103C07CF1B9D7800E6D1996
:102BD200006E800E005C02E16E516C5D21E26C5170
:102BE2006E5D856FBAEC08F000C004F001C005F01C
:102BF20002C006F003C007F073C100F074C101F017
:102C020075C102F076C103F0A5EC0EF000C073F1BD
:102C120001C074F102C075F103C076F16CC16EF1AE
:102C2200050E01016C25006E000E6D21016E005033
:102C32006F5F0150705B6C516D1103E172B701D08F
:102C420004D0010E6F5F000E705B030E7115006EF3
:102C520072C101F0000E01160050011004E0010ED5
:102C62006F5F000E705B71A539D071A312D071A194
:102C720003D02D0E646F02D02B0E646F5DC1E1FF95
:102C82005EC1E2FF64C1E6FF5D4B5E2B7D4B7E2B96
:102C92000CD071A10AD05DC1E1FF5EC1E2FF200E3E
:102CA200E66E5D4B5E2B7D4B7E2B800E006E800EA2
:102CB2007019005C02E16F5100080FE25DC1E1FF93
:102CC2005EC1E2FF300EE66E5D4B5E2B7D4B7E2BCE
:102CD200010E6F5F000E705BE8D73AD071B718D063
:102CE200800E006E800E7019005C02E16F510008C8
:102CF2000FE25DC1E1FF5EC1E2FF200EE66E5D4BB9
:102D02005E2B7D4B7E2B010E6F5F000E705BE8D752
:102D120071A312D071A103D02D0E656F02D02B0EBC
:102D2200656F5DC1E1FF5EC1E2FF65C1E6FF5D4B1C
:102D32005E2B7D4B7E2B0CD071A10AD05DC1E1FFD1
:102D42005EC1E2FF200EE66E5D4B5E2B7D4B7E2B5D
:102D520073C100F074C101F075C102F076C103F0D5
:102D6200E1EC0DF000C079F101C07AF102C07BF113
:102D720003C07CF16EC100F0000E016E026E036EA4
:102D820000360090013602360336003600900136D6
:102D920002360336970E0024F66E560E0120F76EA9
:102DA200000E0220F86E0900F5CF04F00900F5CFFD
:102DB20005F00900F5CF06F00900F5CF07F079C15B
:102DC20000F07AC101F07BC102F07CC103F0EBECB0
:102DD2000BF0300E00265DC1E1FF5EC1E2FF00C0D4
:102DE200E6FF5D4B5E2B7D4B7E2B6C516D1103E13B
:102DF20072B701D06FD05DC1E1FF5EC1E2FF2E0E5E
:102E0200E66E5D4B5E2B7D4B7E2B6E516C5F000E32
:102E12006D5B6E534DE06E076EC100F0000E016EE9
:102E2200026E036E0036009001360236033600361B
:102E32000090013602360336970E0024F66E560EC7
:102E42000120F76E000E0220F86E0900F5CF04F0A3
:102E52000900F5CF05F00900F5CF06F00900F5CF1E
:102E620007F079C100F07AC101F07BC102F07CC1A8
:102E720003F0EBEC0BF00A0E046E000E056E066E0C
:102E8200076EEBEC0BF008C000F009C001F00AC0BD
:102E920002F00BC003F0300E00265DC1E1FF5EC1FF
:102EA200E2FF00C0E6FF5D4B5E2B7D4B7E2BB1D770
:102EB2006C516D110FE05DC1E1FF5EC1E2FF300EAA
:102EC200E66E5D4B5E2B7D4B7E2B010E6C5F000E22
:102ED2006D5BEED771AB0BD05DC1E1FF5EC1E2FF6E
:102EE200450EE66E5D4B5E2B7D4B7E2B0AD05DC19F
:102EF200E1FF5EC1E2FF650EE66E5D4B5E2B7D4B30
:102F02007E2B800E7819006E800E005C02E1000EAE
:102F1200775D11E277510008776F7851000E78578C
:102F22005DC1E1FF5EC1E2FF2D0EE66E5D4B5E2BE1
:102F32007D4B7E2B0AD05DC1E1FF5EC1E2FF2B0E0D
:102F4200E66E5D4B5E2B7D4B7E2B0A0E046E000EF1
:102F5200056E77C100F078C101F061EC0DF0300E22
:102F620000265DC1E1FF5EC1E2FF00C0E6FF010194
:102F72005D4B5E2B7D4B7E2B0A0E046E000E056EA2
:102F820077C100F078C101F061EC0DF008C000F0EB
:102F920009C001F0300E00265DC1E1FF5EC1E2FF13
:102FA20000C0E6FF01015D4B5E2B7D4B7E2B71A7BE
:102FB2001AD0800E006E800E7019005C02E16F5113
:102FC200000811E25DC1E1FF5EC1E2FF200EE66E84
:102FD2005D4B5E2B7D4B7E2B010E6F5F000E705B97
:102FE2006F517011EFE116EF10F072A3F3D0800E63
:102FF2007819006E800E005C02E1000E775D0AE235
:10300200010E775D006E000E7859016E00506C5F04
:1030120001506D5B73C100F074C101F075C102F023
:1030220076C103F0E1EC0DF000C079F101C07AF154
:1030320002C07BF103C07CF1010E6E6F6E510A0A71
:1030420034E06EC100F0000E016E026E036E0036B7
:103052000090013602360336003600900136023601
:103062000336970E0024F66E560E0120F76E000E00
:103072000220F86E0900F5CF01F00900F5CF02F049
:103082000900F5CF03F00900F5CF04F004507C5D90
:1030920008E103507B5D05E102507A5D02E10150D7
:1030A200795D01E202D06E2BC9D76E516C5D836FE0
:1030B200000E6D59846F83C16CF184C16DF179C1C9
:1030C20000F07AC101F07BC102F07CC103F098EC00
:1030D2000BF000C004F001C005F002C006F003C00E
:1030E20007F073C100F074C101F075C102F076C13E
:1030F20003F0E7EC0BF000C07FF101C080F102C0E9
:1031020081F103C082F183C185F1BAEC08F07FC17D
:1031120004F080C105F081C106F082C107F004EC21
:1031220002F0000E046E000E056E000E066E7E0E9C
:10313200076E2BEC03F0E1EC0DF000C079F101C059
:103142007AF102C07BF103C07CF16C516D1142E057
:103152000A0E046E000E056E066E076E79C100F04F
:103162007AC101F07BC102F07CC103F0EBEC0BF001
:1031720008C000F009C001F00AC002F00BC003F061
:10318200000E046E031808E10450021805E1045011
:10319200011802E10050000A1DE10A0E046E000E41
:1031A200056E066E076E79C100F07AC101F07BC12F
:1031B20002F07CC103F0EBEC0BF000C079F101C02E
:1031C2007AF102C07BF103C07CF1010E6C5F000E4C
:1031D2006D5BBBD7800E006E800E6D19005C02E144
:1031E2006C510C0816E36CC185F1BBEC06F073C19F
:1031F20004F074C105F075C106F076C107F02BEC3E
:1032020003F000C073F101C074F102C075F103C094
:1032120076F173C100F074C101F075C102F076C19C
:1032220003F0046A056A066A076A3CEC08F0000EBD
:10323200D8A4010E006E0052D8B477D073C100F04A
:1032420074C101F075C102F076C103F0E1EC0DF03A
:10325200000E046E031808E10450021805E1045040
:10326200011802E10050000A60E1800E006E800E3B
:103272007819005C02E17751010857E277C185F1C4
:10328200BAEC08F000C004F001C005F002C006F07C
:1032920003C007F073C100F074C101F075C102F000
:1032A20076C103F0A5EC0EF05F0E046E700E056E93
:1032B200090E066E810E076E53EC08F0010ED8B0AF
:1032C200000E006E005206E0090E0101775F000E4B
:1032D200785B05D00101080E775F000E785B77C13D
:1032E20085F1BAEC08F000C004F001C005F002C09C
:1032F20006F003C007F073C100F074C101F075C19C
:1033020002F076C103F0A5EC0EF0E1EC0DF000C086
:1033120079F101C07AF102C07BF103C07CF10101B5
:10332200736B746B756B766B38D073C100F074C1BC
:1033320001F075C102F076C103F0E1EC0DF000C0BE
:1033420079F101C07AF102C07BF103C07CF179C14D
:1033520000F07AC101F07BC102F07CC103F098EC6D
:103362000BF000C004F001C005F002C006F003C07B
:1033720007F073C100F074C101F075C102F076C1AB
:1033820003F0E7EC0BF000C073F101C074F102C06E
:1033920075F103C076F1776B786B010E6E6F6E512B
:1033A2000A0A34E06EC100F0000E016E026E036E76
:1033B20000360090013602360336003600900136A0
:1033C20002360336970E0024F66E560E0120F76E73
:1033D200000E0220F86E0900F5CF01F00900F5CFCA
:1033E20002F00900F5CF03F00900F5CF04F0045014
:1033F2007C5D08E103507B5D05E102507A5D02E1EC
:103402000150795D01E202D06E2BC9D76E516C2555
:10341200006E000E6D21016E775100267851012257
:1034220000506F5F0150705B72B704D06C516D1128
:1034320001E104D0010E6F5F000E705B030E711587
:10344200006E72C101F0000E01160050011004E07E
:10345200010E6F5F000E705B71A539D071A312D09F
:1034620071A103D02D0E666F02D02B0E666F5DC167
:10347200E1FF5EC1E2FF66C1E6FF5D4B5E2B7D4B65
:103482007E2B0CD071A10AD05DC1E1FF5EC1E2FFCB
:10349200200EE66E5D4B5E2B7D4B7E2B800E006E0A
:1034A200800E7019005C02E16F5100080FE25DC1ED
:1034B200E1FF5EC1E2FF300EE66E5D4B5E2B7D4B9F
:1034C2007E2B010E6F5F000E705BE8D73AD071B7AA
:1034D20018D0800E006E800E7019005C02E16F51F0
:1034E20000080FE25DC1E1FF5EC1E2FF200EE66E61
:1034F2005D4B5E2B7D4B7E2B010E6F5F000E705B72
:10350200E8D771A312D071A103D02D0E676F02D03C
:103512002B0E676F5DC1E1FF5EC1E2FF67C1E6FF8F
:103522005D4B5E2B7D4B7E2B0CD071A10AD05DC111
:10353200E1FF5EC1E2FF200EE66E5D4B5E2B7D4B2E
:103542007E2B6EC100F06E0700524CE06EC100F09F
:10355200000E016E026E036E0036009001360236D6
:10356200033600360090013602360336970E0024E9
:10357200F66E560E0120F76E000E0220F86E09005C
:10358200F5CF04F00900F5CF05F00900F5CF06F0FC
:103592000900F5CF07F079C100F07AC101F07BC1D3
:1035A20002F07CC103F0EBEC0BF00A0E046E000E8D
:1035B200056E066E076EEBEC0BF008C000F009C05A
:1035C20001F00AC002F00BC003F0300E00265DC10C
:1035D200E1FF5EC1E2FF00C0E6FF5D4B5E2B7D4B6B
:1035E2007E2BAFD7800E006E800E7819005C02E150
:1035F200775100080FE25DC1E1FF5EC1E2FF300ECC
:10360200E66E5D4B5E2B7D4B7E2B010E775F000ECF
:10361200785BE8D7800E000A006E800E6D19005CA0
:1036220002E16C51080803E2080E6E6F02D06CC111
:103632006EF16E516C5F000E6D5B6E5303E172B7FB
:1036420001D00AD05DC1E1FF5EC1E2FF2E0EE66E3F
:103652005D4B5E2B7D4B7E2B6EC185F1BAEC08F083
:1036620073C104F074C105F075C106F076C107F0AC
:1036720004EC02F017EC06F000C079F101C07AF117
:1036820002C07BF103C07CF16E534DE06E076EC148
:1036920000F0000E016E026E036E003600900136DD
:1036A2000236033600360090013602360336970E94
:1036B2000024F66E560E0120F76E000E0220F86E00
:1036C2000900F5CF04F00900F5CF05F00900F5CFA8
:1036D20006F00900F5CF07F079C100F07AC101F0D8
:1036E2007BC102F07CC103F0EBEC0BF00A0E046E1E
:1036F200000E056E066E076EEBEC0BF008C000F0D4
:1037020009C001F00AC002F00BC003F0300E00261F
:103712005DC1E1FF5EC1E2FF00C0E6FF5D4B5E2BD3
:103722007D4B7E2BB1D76C516D110FE05DC1E1FF76
:103732005EC1E2FF300EE66E5D4B5E2B7D4B7E2B53
:10374200010E6C5F000E6D5BEED771A71AD0800E72
:10375200006E800E7019005C02E16F51000811E2E8
:103762005DC1E1FF5EC1E2FF200EE66E5D4B5E2BA6
:103772007D4B7E2B010E6F5F000E705B6F517011DF
:10378200EFE116EF10F0C00E7115016E72C102F07A
:10379200000E0216000E021802E1000E0118D8A453
:1037A20080D071A927D062C1E9FF63C1EAFFEECFE1
:1037B20000F0EECF01F000C0E9FF01C0EAFFEECF5A
:1037C20079F1EECF7AF1EECF7BF1EECF7CF162C1EF
:1037D200E9FF63C1EAFF040EEE24006E000EEE2044
:1037E200016E62C1E1FF63C1E2FF00C0E6FF01C0FA
:1037F200E6FF2FD062C1E9FF63C1EAFFEECF00F01E
:10380200EECF01F000C0E9FF01C0EAFFEECF00F009
:10381200EECF01F0000E01BEFF0E026E036E00C07D
:1038220079F101C07AF102C07BF103C07CF162C17F
:10383200E9FF63C1EAFF020EEE24006E000EEE20E5
:10384200016E62C1E1FF63C1E2FF00C0E6FF01C099
:10385200E6FF800E7C19006E800E005C08E1000E0F
:103862007B5D05E1000E7A5D02E1000E795D18E2F2
:10387200030E7113000E7213006A016A026A036A70
:103882007951005E7A51015A7B51025A7C51035A96
:1038920000C079F101C07AF102C07BF103C07CF172
:1038A2004ED071A927D062C1E9FF63C1EAFFEECF12
:1038B20000F0EECF01F000C0E9FF01C0EAFFEECF59
:1038C20079F1EECF7AF1EECF7BF1EECF7CF162C1EE
:1038D200E9FF63C1EAFF040EEE24006E000EEE2043
:1038E200016E62C1E1FF63C1E2FF00C0E6FF01C0F9
:1038F200E6FF25D062C1E9FF63C1EAFFEECF00F027
:10390200EECF01F000C0E9FF01C0EAFFEECF79F18E
:10391200EECF7AF1000E7B6F7C6F62C1E9FF63C16B
:10392200EAFF020EEE24006E000EEE20016E62C16E
:10393200E1FF63C1E2FF00C0E6FF01C0E6FF000E47
:103942006D1902E1000E6C190FE1000E006E7C1978
:1039520008E100507B1905E100507A1902E1795122
:10396200000A02E16C4B6D2BC00E7115006E00C097
:1039720005F0AED0010E6E6F6E510A0A34E06EC1D0
:1039820000F0000E016E026E036E003600900136EA
:103992000236033600360090013602360336970EA1
:1039A2000024F66E560E0120F76E000E0220F86E0D
:1039B2000900F5CF01F00900F5CF02F00900F5CFBB
:1039C20003F00900F5CF04F004507C5D08E10350D8
:1039D2007B5D05E102507A5D02E10150795D01E211
:1039E20002D06E2BC9D782D0010E6E6F6E51080ABB
:1039F20034E06EC100F0000E016E026E036E0036FE
:103A02000090013602360336003600900136023647
:103A12000336E50E0024F66E560E0120F76E000EF8
:103A22000220F86E0900F5CF01F00900F5CF02F08F
:103A32000900F5CF03F00900F5CF04F004507C5DD6
:103A420008E103507B5D05E102507A5D02E101501D
:103A5200795D01E202D06E2BC9D748D0010E6E6F9C
:103A62006E510C0A34E06EC100F0000E016E026E5F
:103A7200036E00360090013602360336003600909F
:103A8200013602360336670E0024F66E560E01200A
:103A9200F76E000E0220F86E0900F5CF01F0090062
:103AA200F5CF02F00900F5CF03F00900F5CF04F0DD
:103AB20004507C5D08E103507B5D05E102507A5DB4
:103AC20002E10150795D01E202D06E2BC9D70ED01E
:103AD2000550000AD8B44ED70550C00AD8B44AD708
:103AE2000550800A81E00550400AB8E0800E006E61
:103AF200800E6D19005C02E16C516E5D03E26CC1D7
:103B02006EF10DD0800E6D19006E800E005C02E128
:103B12006E516C5D04E26EC16CF1000E6D6F6F51FF
:103B220070110EE0030E7115006E72C101F0000EED
:103B320001160050011004E0010E6F5F000E705B71
:103B4200800E6D19006E800E7019005C02E16F51DB
:103B52006C5D05E26C516F5F6D51705B02D06F6BF3
:103B6200706BC40E7115016E7251080B026E025019
:103B7200080A02E1400E011808E16F51701104E0D9
:103B8200010E6F5F000E705B1CD0C00E7115016ECE
:103B92007251080B026E0250080A02E1800E0118EF
:103BA20010E1800E006E800E7019005C02E16F5110
:103BB200020805E2020E6F5F000E705B02D06F6BAF
:103BC200706B71A55DD071A312D071A103D02D0EBF
:103BD200686F02D02B0E686F5DC1E1FF5EC1E2FF2C
:103BE20068C1E6FF5D4B5E2B7D4B7E2B34D071A10D
:103BF2000BD05DC1E1FF5EC1E2FF200EE66E5D4BC0
:103C02005E2B7D4B7E2B27D0C00E7115016E72513B
:103C1200080B026E0250080A02E1800E01181BE135
:103C22005DC1E1FF5EC1E2FF300EE66E5D4B5E2BD1
:103C32007D4B7E2B71AB03D0580E696F02D0780E8C
:103C4200696F5DC1E1FF5EC1E2FF69C1E6FF5D4BE5
:103C52005E2B7D4B7E2B6F51701111E05DC1E1FF38
:103C62005EC1E2FF300EE66E5D4B5E2B7D4B7E2B1E
:103C7200010E6F5F000E705B6F517011EFE174D037
:103C82006F51701113E071B711D05DC1E1FF5EC1D8
:103C9200E2FF200EE66E5D4B5E2B7D4B7E2B010E0E
:103CA2006F5F000E705B6F517011EFE171A312D064
:103CB20071A103D02D0E6A6F02D02B0E6A6F5DC107
:103CC200E1FF5EC1E2FF6AC1E6FF5D4B5E2B7D4B09
:103CD2007E2B0CD071A10AD05DC1E1FF5EC1E2FF73
:103CE200200EE66E5D4B5E2B7D4B7E2BC00E71155A
:103CF200016E7251080B026E0250080A02E1400E78
:103D020001180BE15DC1E1FF5EC1E2FF300EE66E1C
:103D12005D4B5E2B7D4B7E2B27D0C00E7115016E45
:103D22007251080B026E0250080A02E1800E01185D
:103D32001BE15DC1E1FF5EC1E2FF300EE66E5D4B4D
:103D42005E2B7D4B7E2B71AB03D0580E6B6F02D076
:103D5200780E6B6F5DC1E1FF5EC1E2FF6BC1E6FFF2
:103D62005D4B5E2B7D4B7E2B800E006E800E6D199F
:103D7200005C02E16C516E5D0BE25DC1E1FF5EC170
:103D8200E2FF300EE66E5D4B5E2B7D4B7E2BECD759
:103D92006CC100F06DC101F0010E6C5F000E6D5B35
:103DA20000500110D8B42AD1C00E7115006E00C0A7
:103DB2007FF10AD16CC100F06DC101F0000E6DBF40
:103DC200FF0E026E036E0036009001360236033695
:103DD20000360090013602360336970E0024F66E46
:103DE200560E0120F76E000E0220F86E0900F5CF84
:103DF20004F00900F5CF05F00900F5CF06F009003F
:103E0200F5CF07F079C100F07AC101F07BC102F071
:103E12007CC103F0EBEC0BF00A0E046E000E056E93
:103E2200066E076EEBEC0BF008C000F009C001F063
:103E32000AC002F00BC003F0300E00246E6FD3D024
:103E420071AB45D06CC100F06DC101F0000E6DBFC9
:103E5200FF0E026E036E0036009001360236033604
:103E620000360090013602360336E50E0024F66E67
:103E7200560E0120F76E000E0220F86E0900F5CFF3
:103E820004F00900F5CF05F00900F5CF06F00900AE
:103E9200F5CF07F079C100F07AC101F07BC102F0E1
:103EA2007CC103F0EBEC0BF00F0E0016000E0116B6
:103EB20002160316960E0024F66E570E0120F76EB8
:103EC200000E0220F86E0900F5CF6EF144D06CC1ED
:103ED20000F06DC101F0000E6DBFFF0E026E036EA9
:103EE2000036009001360236033600360090013665
:103EF20002360336E50E0024F66E560E0120F76EEA
:103F0200000E0220F86E0900F5CF04F00900F5CF8B
:103F120005F00900F5CF06F00900F5CF07F079C1E9
:103F220000F07AC101F07BC102F07CC103F0EBEC3E
:103F32000BF00F0E0016000E011602160316A70E46
:103F42000024F66E570E0120F76E000E0220F86E66
:103F52000900F5CF6EF147D06CC100F06DC101F0E0
:103F6200000E6DBFFF0E026E036E0036009001362A
:103F72000236033600360090013602360336670EEB
:103F82000024F66E560E0120F76E000E0220F86E27
:103F92000900F5CF04F00900F5CF05F00900F5CFCF
:103FA20006F00900F5CF07F079C100F07AC101F0FF
:103FB2007BC102F07CC103F0EBEC0BF0070E0014A6
:103FC2006E6F300E6E270FD07F51000AD8B4F2D632
:103FD2007F51C00AD8B4EED67F51800AD8B430D708
:103FE2007F51400AB9E05DC1E1FF5EC1E2FF6EC1EF
:103FF200E6FF5D4B5E2B7D4B7E2BCAD671A71AD096
:10400200800E006E800E7019005C02E16F51000894
:1040120011E25DC1E1FF5EC1E2FF200EE66E5D4B83
:104022005E2B7D4B7E2B010E6F5F000E705B6F511E
:104032007011EFE116EF10F07DC100F07EC101F0CA
:0240420012006A
:104044005DC100F00032009E0032009E0032009EEE
:104054000032009EB80E0024F66E570EF76E000E66
:10406400F722000EF86E000EF8220900F5CF00F0DA
:104074005EC1E1FF5FC1E2FF00C0E6FF010E010186
:104084005E25E16E000E5F21E26E0F0E5D15006E7F
:10409400B80E0024F66E570EF76E000EF722000ECF
:1040A400F86E000EF8220900F5CF00F000C0E6FF1C
:1040B400020E5E25E16E000E5F21E26EE66A1200DA
:1040C400F00E01015D15026E02C000F00032009E88
:1040D4000032009E0032009E0032009E008E008C52
:1040E40000C05EF182C085F1100E0010866FC5EC31
:1040F4000DF000C083F0000E0001846F1A0E0D6EE7
:104104000D2EFED7000082C085F1EF0E01015E1571
:10411400866FC5EC0DF000C083F0000E0001846FC3
:104124001A0E0D6E0D2EFED700000F0E01015D1547
:10413400006E008E008C00C05EF182C085F1100E0E
:104144000010866FC5EC0DF000C083F0000E000176
:10415400846F1A0E0D6E0D2EFED7000082C085F1FD
:10416400EF0E01015E15866FC5EC0DF000C083F003
:10417400000E0001846F1A0E0D6E0D2EFED7000086
:02418400120027
:104186000001836B846BF00E01015D15026E02C0A7
:1041960000F00032009E0032009E0032009E003287
:1041A600009E008E00C05FF182C085F1100E0010E7
:1041B600866FC5EC0DF000C083F0000E0001846F21
:1041C600350E0D6E0D2EFED782C085F1EF0E010164
:1041D6005F15866FC5EC0DF000C083F0000E000180
:1041E600846F350E0D6E0D2EFED701015E532DE048
:1041F6000F0E5D15006E008E00C05FF182C085F166
:10420600100E0010866FC5EC0DF000C083F0000E96
:104216000001846F0A0E0D6E0D2EFED7000082C0BF
:1042260085F1EF0E01015F15866FC5EC0DF000C03C
:1042360083F0000E0001846F680E0C6EE40E0D6EA6
:0C4246000D2EFED70C2EFCD7000012003D
:104252000D0E0101906F9DEC00F00A0E0101906FAE
:064262009DEC00F01200CB
:104268000101606B030E605D0AE260515E25E16E3C
:10427800000E5F21E26E200EE66E602BF3D76051D0
:104288005E25E16E000E5F21E26EE66A600760510E
:104298005E25616F000E5F21626F0A0E046E5DC1BC
:1042A80000F094EC02F008C000F0300E002661C166
:1042B800E1FF62C1E2FF00C0E6FF0A0E046E5DC1C5
:1042C80000F094EC02F000C05DF10050000A01E13A
:0842D80002D06007DCD71200E0
:1042E0005FC1F6FF60C1F7FF61C1F8FF0900F5CFBC
:1042F00000F0005218E05FC1F6FF60C1F7FF61C136
:10430000F8FF0900F5CF00F05DC1E1FF5EC1E2FFFB
:1043100000C0E6FF01015D4B5E2B010E5F27000E22
:1043200060236123DDD75DC1E1FF5EC1E2FFE66A84
:02433000120079
:10433200A69C5EC1AAFF5DC1A9FFA69EA680A8CFCA
:0443420000F0120075
:104346005DC104F05EC105F004C0E9FF05C0EAFFE7
:10435600EE5203E0044A052AF7D704C002F005C06E
:1043660003F0044A052A5FC100F060C101F00101B3
:104376005F4B602B00C0E9FF01C0EAFF02C0E1FF0E
:1043860003C0E2FFEECFE6FF02C0E9FF03C0EAFF8B
:10439600EE5201E0E2D75DC100F05EC101F012000D
:0E43A6007EC000F07FC001F0C7EC00F01200F6
:1043B4000101606B5DC1E9FF5EC1EAFFEECF5FF111
:1043C4005F51000A0FE05FC190F19DEC00F0010124
:1043D400602B60515D25E96E000E5E21EA6EEECF22
:0643E4005FF1EED71200AC
:1043EA004B0E01014F6F010E506F46C15DF147C17F
:1043FA005EF148C15FF149C160F14AC161F14F0EF6
:10440A00626F010E636F11EC10F000C04DF101C034
:10441A004EF100504625E16E01504721E26EE66AF0
:0A442A004DC100F04EC101F0120078
:10443400C280C19EC08EC08AC088C096C082C0940B
:0C444400C090C196C194C192C1901200BA
:10445000520E0B6E2B0E0C6E000E0D6E0D2EFED737
:0C4460000C2EFCD70B2EFAD70000120027
:10446C000101496B4A6B46C1F6FF47C1F7FF48C1D2
:10447C00F8FF0900F5CF01F00150000A1CE0800E96
:10448C004A19006E800E005C02E1100E495D13E2C9
:10449C0046C1F6FF47C1F7FF48C1F8FF0900F5CF49
:1044AC005DF10ADE010E01014627000E4723482369
:0844BC00494B4A2BD8D712002E
:1044C4000101496B4A6B46C1F6FF47C1F7FF48C17A
:1044D400F8FF0900F5CF00F000520CE0800E4A19F5
:1044E400006E800E005C02E1100E495D03E2494B50
:1044F4004A2BE9D746C1F6FF47C1F7FF48C1F8FF89
:104504000900F5CF5DF1DCDD010E01014627000E47
:06451400472348231200BA
:10451A0001014C51000805E3070E4D6F000E4E6F66
:10452A0012D04C51160805E2170E4F6F000E506F4D
:10453A0006D04C51010F4F6F506B000E50234FC1E4
:10454A004DF150C14EF14DC157F14EC158F1516B69
:10455A00526B046A056A066A076A46C100F047C1D7
:10456A0001F048C102F049C103F053EC08F0010E12
:10457A00D8B0000E006E005209E04AC1E1FF4BC1FB
:10458A00E2FF2D0EE66E4A4B4B2B487F46C104F0E4
:10459A0047C105F048C106F049C107F0006A016A3F
:1045AA00026A036A53EC08F0010ED8B0000E006EDE
:1045BA00005237E0000E046E000E056E000E066E05
:1045CA007F0E076E46C100F047C101F048C102F0F4
:1045DA0049C103F053EC08F0010ED8B0000E006E8A
:1045EA0000521FE046C100F047C101F048C102F085
:1045FA0049C103F0000E046E000E056E200E066E11
:10460A00820E076E04EC02F000C046F101C047F1C9
:10461A0002C048F103C049F1010E515F000E525B1E
:10462A00C9D7000E046E000E056E200E066E820EAD
:10463A00076E46C100F047C101F048C102F049C106
:10464A0003F053EC08F0000ED8B0010E006E0052D1
:10465A001EE0000E046E000E056E200E066E820E1F
:10466A00076E46C100F047C101F048C102F049C1D6
:10467A0003F0A5EC0EF000C046F101C047F102C0FC
:10468A0048F103C049F10101514B522BCAD751518C
:10469A00572752515823010E536F000E546F000EC4
:1046AA00596F000E5A6F000E5B6F7F0E5C6F800EA3
:1046BA005419006E800E5819005C02E15751535D7F
:1046CA001EE2000E046E000E056E200E066E820EAD
:1046DA00076E59C100F05AC101F05BC102F05CC11A
:1046EA0003F0A5EC0EF000C059F101C05AF102C066
:1046FA005BF103C05CF10101534B542BD8D7000E78
:10470A00046E000E056E000E066E800E076E59C10D
:10471A0000F05AC101F05BC102F05CC103F0A5ECE4
:10472A000EF046C104F047C105F048C106F049C180
:10473A0007F02BEC03F000C046F101C047F102C0BC
:10474A0048F103C049F1000E046E000E056E200EFA
:10475A00066E820E076E53EC08F0000ED8B0010EFA
:10476A00006E00520BE0000E0101466F000E476F0B
:10477A00000E486F7F0E496F514B522B0101800E7C
:10478A005219006E800E005C02E1000E515D38E2A3
:10479A004AC1E1FF4BC1E2FF300EE66E4A4B4B2B9A
:1047AA004AC1E1FF4BC1E2FF2E0EE66E4A4B4B2B8C
:1047BA00800E5819006E800E005C02E1000E575DF3
:1047CA0004E25751515F5851525BFF0E536FFF0E6F
:1047DA00546F800E5219006E800E5419005C02E16B
:1047EA005351515D0DE24AC1E1FF4BC1E2FF300E68
:1047FA00E66E4A4B4B2B010E535F000E545BE9D712
:10480A00536B546B800E5419006E800E5819005C5D
:10481A0002E15751535D63E246C100F047C101F01E
:10482A0048C102F049C103F063EC0FF000C055F132
:10483A0001C056F1300E00264AC1E1FF4BC1E2FF2A
:10484A0000C0E6FF4A4B4B2B5451521902E1515119
:10485A00531908E14AC1E1FF4BC1E2FF2E0EE66E91
:10486A004A4B4B2B55C100F056C101F0CDEC0FF06D
:10487A0000C059F101C05AF102C05BF103C05CF1FA
:10488A0000C004F001C005F002C006F003C007F042
:10489A0046C100F047C101F048C102F049C103F026
:1048AA00E7EC0BF000C046F101C047F102C048F145
:1048BA0003C049F1000E046E000E056E200E066E4E
:1048CA00820E076E04EC02F000C046F101C047F107
:1048DA0002C048F103C049F1534B542B93D74AC144
:0A48EA00E1FF4BC1E2FFE66A120095
:1048F4000101486B496B46C1E9FF47C1EAFFEE502D
:10490400000A17E0800E4919006E800E005C02E177
:10491400100E485D0EE246C1E9FF47C1EAFFEECF43
:104924005DF162EC20F00101464B472B484B492BCB
:04493400E2D71200B4
:10493800830EC21646C100F0003600900036009083
:104948000050C2120CEC10F0C282C2A201D0FDD7F6
:10495800C4CF01F0006A00C047F101C048F1C3505C
:104968000012000E011200C047F101C048F1000E0C
:104978000014026E0150800B036E000E031802E152
:10498800000E021803E00101476B486B47C100F0B5
:0649980048C101F012000D
:10499E007A0E0B6EC10E0C6E810E0D6E0D2EFED7A5
:1049AE000C2EFCD70B2EFAD700000000300E0101A2
:1049BE005D6F5E6BC3EC20F0050E0B6E0F0E0C6E72
:1049CE00F10E0D6E0D2EFED70C2EFCD70B2EFAD738
:1049DE00300E01015D6F5E6BC3EC20F0020E0B6EAC
:1049EE00A00E0C6E920E0D6E0D2EFED70C2EFCD759
:1049FE000B2EFAD70000300E01015D6F5E6BC3EC1B
:104A0E0020F0020E0B6EA00E0C6E920E0D6E0D2E81
:104A1E00FED70C2EFCD70B2EFAD70000200E01016C
:104A2E005D6F5E6BC3EC20F0020E0B6EA00E0C6E73
:104A3E00920E0D6E0D2EFED70C2EFCD70B2EFAD726
:104A4E000000280E01015D6F010E5E6FC3EC20F0B9
:104A5E00020E0B6EA00E0C6E920E0D6E0D2EFED76C
:104A6E000C2EFCD70B2EFAD70000080E01015D6F3D
:104A7E00010E5E6FC3EC20F0020E0B6EA00E0C6EDC
:104A8E00920E0D6E0D2EFED70C2EFCD70B2EFAD7D6
:104A9E000000010E01015D6F010E5E6FC3EC20F090
:104AAE00090E0B6E1E0E0C6EE40E0D6E0D2EFED745
:104ABE000C2EFCD70B2EFAD70000060E01015D6FEF
:104ACE00010E5E6FC3EC20F0020E0B6EA00E0C6E8C
:104ADE00920E0D6E0D2EFED70C2EFCD70B2EFAD786
:104AEE0000000C0E01015D6F010E5E6FC3EC20F035
:104AFE00020E0B6EA00E0C6E920E0D6E0D2EFED7CC
:0C4B0E000C2EFCD70B2EFAD70000120072
:104B1A003A0E0101306F010E316F900E326F010EA5
:104B2A00336FFF0E346FFF0E356F000E366F000EB7
:104B3A00376FFF0E246FFF0E256F000E266F000ED3
:104B4A00276FFF0E286FFF0E296F000E2A6F000EC7
:104B5A002B6FAC8A900EAB6E948E949C9EAA03D057
:084B6A00AECF00F0FBD71200F2
:104B7200FF0E816E830E936E0F01396B070E806EEE
:104B8200386B388138832F0E926E806A928A826ADD
:104B92003A6BFF0E946E94869488948E949C606A0D
:024BA2001200FF
:104BA4000900F5CFE6FF0006FBE10106F9E112007A
:104BB40046C102F047C103F002C000F003C001F097
:104BC400024A032A00C0E9FF01C0EAFFEE5201E0F5
:104BD400F3D701014651025C006E47510358016E40
:0A4BE400010E005E000E015A1200DF
:104BEE0001014A6B496B4751000825E228C05DF16F
:104BFE0029C05EF1FA0E5F6F570E606F000E616F87
:104C0E0070EC21F046C15DF15A0E01015E6F000E8F
:104C1E005F6F34EC21F028C05DF129C05EF15A0EB1
:104C2E005F6F000E606FA3EC21F028C05DF129C00C
:104C3E005EF1DAEC21F0C69E3EEC05F046C18AF13B
:104C4E0088EC05F000C048F1000E016EFF0E011851
:104C5E0002E1FF0E001803E1C9CF48F1C69ED3EC66
:104C6E0021F001014851000A0DE0496B475100083F
:104C7E0008E2EF0E5D6F570E5E6F000E5F6FEEEC8B
:104C8E000FF054D0010E0101496F4E0EE16E000E71
:104C9E00E26E4A51E126D8B0E22AE1CFE1FFE2CF3F
:104CAE00E2FF46C1E6FF475100083EE2090E906F53
:104CBE009DEC00F05A0E01015D6F000E5E6F050E49
:104CCE005F6F570E606F000E616F70EC21F0300E4B
:104CDE0001011C250001636F46C15DF16E0E0101DD
:104CEE005E6F000E5F6F34EC21F05A0E5D6F000E9A
:104CFE005E6FDAEC21F0040E5D6F580E5E6F000EE3
:104D0E005F6FEEEC0FF046C15DF15A0E01015E6F62
:104D1E00000E5F6F22EC20F05A0E5D6F000E5E6F7C
:104D2E00DAEC21F029EC21F001014A2BFCEC01F028
:104D3E00050E0B6E0F0E0C6EF10E0D6E0D2EFED7B8
:104D4E000C2EFCD70B2EFAD7D3EC00F00050000A35
:104D5E0001E1FAD701014751000802E229EC21F0E6
:064D6E0049C100F0120033
:104D7400A60E0101386F010E396F000E3A6F000E56
:104D84003B6F7C0E00017A6F0A0E7B6F000E7C6F06
:104D9400000E7D6F000E4A6E060E4B6E000E4C6EBA
:104DA400000E4D6EFF0E0101206FFF0E216FFF0EEE
:104DB400226FFF0E236F100E0001CF6F0B0ED06F0A
:104DC4008A0ED16F010ED26FF80E7E6F030E7F6FC5
:104DD400000E806F000E816F949894968B988B963A
:0E4DE40094889486C79EC79C380EC66E120037
:104DF20046C148F147C149F148C15DF149C15EF17F
:104E020099EC21F000C04AF1000E01014B6F000E37
:104E12004B1902E1000E4A1901E133D0800E030A58
:104E2200006E800E4919005C02E14851FF0801E260
:104E320028D04AC190F19DEC00F001014651485D35
:104E4200006E47514959016E2A0E0024E16E000E90
:104E52000120E26EE1CFE1FFE2CFE2FF4AC1E6FFCD
:104E6200680E0C6EE40E0D6E0D2EFED70C2EFCD7C6
:104E72000000484B492B000E4B1902E1000E4A1963
:044E8200BBE112007E
:104E860011EC2CF0D38CD38AD3889B8CD392D390FD
:104E96006DDE01011E6B1F6B800E1F19006E800EEA
:104EA600005C02E1400E1E5D0EE2D80E1E25E16E8C
:104EB600000E1F21E26EE1CFE1FFE2CFE2FFE66ADC
:104EC6001E4B1F2BE9D7D80E286E000E296EB8860A
:104ED600B06A8A0EAF6EAC841DDE290E0B6E960E7E
:104EE6000C6E7F0E0D6E0D2EFED70C2EFCD70B2EE4
:104EF600FAD728C046F129C047F159DE00C01CF197
:104F060001C01DF10001D56BD66BD36BD46B29ECB8
:104F160021F029EC21F0840E01015D6F570E5E6FC2
:104F2600000E5F6FEEEC0FF05A0E01015D6F550E2D
:104F36005E6F000E5F6FEEEC0FF028C05DF129C0CA
:104F46005EF1330E01015F6F560E606F000E616FEA
:104F560070EC21F029EC21F028C05DF129C05EF14A
:104F6600DAEC21F0BF0E5D6F560E5E6F000E5F6FBE
:104F7600EEEC0FF00101466B476B38DF29EC21F0B0
:104F8600200E0101466F000E476F30DF29EC21F03D
:104F9600600E0101466F000E476F28DF29EC21F0F5
:104FA600280EC86EE4DE800E0101466F000E476FC4
:104FB6001DDF29EC21F0140E01015D6F550E5E6FA9
:104FC600000E5F6FEEEC0FF001011E6B1F6B800E83
:104FD6001F19006E800E005C02E1080E1E5D0EE2D7
:104FE6004E0E1E25E16E000E1F21E26EE1CFE1FF9F
:104FF600E2CFE2FFE66A1E4B1F2BE9D7200E1E6F9B
:10500600000E1F6F800E1F19006E800E005C02E1FD
:10501600FE0E1E5D18E21EC146F1476BE5DD00C0BF
:10502600D7F0050E0B6E0F0E0C6EF10E0D6E0D2EDB
:10503600FED70C2EFCD70B2EFAD7020E01011E2727
:10504600000E1F23DFD729EC21F0930E01015D6FBF
:10505600550E5E6F000E5F6FEEEC0FF001011C6BDC
:105066001D6B800E1D19006E800E005C02E1080E9D
:105076001C5D41E25A0E5D6F000E5E6F5D0E5F6F46
:10508600570E606F000E616F70EC21F0310E01015A
:105096001C250001636F4E0E01011C25E96E000EF2
:1050A6001D21EA6EE9CFE9FFEACFEAFFEE500008DC
:1050B60013E24E0E1C25E96E000E1D21EA6EE9CFA5
:1050C600E9FFEACFEAFFEECF5DF1690E5E6F000EF3
:1050D6005F6F22EC20F002D00001656B5A0E0101D1
:1050E6005D6F000E5E6FDAEC21F029EC21F0010114
:1050F6001C4B1D2BB6D7400E0001826F4DDC010EF6
:1051060001015D6F010E5E6FC3EC20F0800E0101A0
:105116005D6F010E5E6FC3EC20F0030E0B6E080E82
:105126000C6E770E0D6E0D2EFED70C2EFCD70B2EA9
:10513600FAD7800E01015D6F010E5E6FC3EC20F0A1
:10514600330E0101466F570E476F000E486F36EC5F
:1051560022F0C00E5D6F010E5E6FC3EC20F01E0ED6
:105166000101466F570E476F000E486F36EC22F06E
:1051760028EC22F028EC22F029EC21F0AA0E0101FD
:10518600466F000E476F32DE29EC21F01AEC22F052
:105196000001D56BD66BD80E286E000E296E010E57
:1051A60001015D6F010E5E6FC3EC20F0030E0B6E06
:1051B600080E0C6E770E0D6E0D2EFED70C2EFCD73C
:1051C6000B2EFAD7800E01015D6F010E5E6FC3ECE8
:1051D60020F0110E0101466F580E476F000E486F02
:1051E60062EC22F0C00E5D6F010E5E6FC3EC20F024
:1051F6000B0E0101466F580E476F000E486F62ECAA
:1052060022F0010E5D6F010E5E6FC3EC20F028ECFC
:1052160022F000018D6BCD6BCE6B9E9A9D8AF28C2F
:10522600F28E0101466B9CEC24F000C085F001C0B3
:1052360086F0D80E286E000E296E030E0B6E080E31
:105246000C6E770E0D6E0D2EFED70C2EFCD70B2E88
:10525600FAD728C046F129C047F1D70E0101486F99
:10526600570E496F000E4A6F85C04BF186C04CF150
:10527600F5EC21F028C05DF129C05EF1DAEC21F0F1
:10528600800E5D6F010E5E6FC3EC20F028C046F104
:1052960029C047F17AEC24F01C0E5D6F580E5E6F44
:1052A600000E5F6FEEEC0FF085C000F086C001F0D7
:1052B600CDEC0FF0E50E046EFF0E056E1F0E066EAA
:1052C600770E076E04EC02F000C087F001C088F08C
:1052D60002C089F003C08AF000C046F101C047F160
:1052E60002C048F103C049F15A0E01014A6F000E8F
:1052F6004B6F020E4C6F8DEC22F05A0E5D6F000E56
:105306005E6FDAEC21F03B0E906F9DEC00F0800EA4
:1053160001015D6F010E5E6FC3EC20F028C046F1FF
:1053260029C047F17AEC24F08A0E5D6F010E5E6F9C
:10533600C3EC20F05A0E0101466F000E476F7AEC5F
:1053460024F028EC22F0030E0B6E080E0C6E770E7E
:105356000D6E0D2EFED70C2EFCD70B2EFAD7010E96
:10536600466F9CEC24F000C08BF001C08CF028C086
:1053760046F129C047F1E30E0101486F570E496F08
:10538600000E4A6F00C04BF101C04CF1F5EC21F064
:1053960028C05DF129C05EF1DAEC21F03B0E906F7A
:1053A6009DEC00F0C00E01015D6F010E5E6FC3EC57
:1053B60020F028C046F129C047F17AEC24F0170EF8
:1053C6005D6F580E5E6F000E5F6FEEEC0FF08BC0D8
:1053D60000F08CC001F0CDEC0FF0E50E046EFF0E70
:1053E600056E1F0E066E770E076E04EC02F000C007
:1053F6002CF101C02DF102C02EF103C02FF100C027
:1054060046F101C047F102C048F103C049F15A0E06
:1054160001014A6F000E4B6F020E4C6F8DEC22F0AD
:105426005A0E5D6F000E5E6FDAEC21F029EC21F06A
:10543600CA0E01015D6F010E5E6FC3EC20F05A0EBD
:105446000101466F000E476F7AEC24F0520E0B6E88
:105456002B0E0C6E000E0D6E0D2EFED70C2EFCD7ED
:105466000B2EFAD70000000E411902E1010E401979
:105476004CE100018D51550A48E19F51230A45E14F
:10548600200EA06F9D6B800E01015D6F010E5E6F99
:10549600C3EC20F0030E0B6E080E0C6E770E0D6E2D
:1054A6000D2EFED70C2EFCD70B2EFAD7720E01014D
:1054B6005D6F570E5E6F000E5F6FEEEC0FF0C00E65
:1054C60001015D6F010E5E6FC3EC20F0030E0B6EE3
:1054D600080E0C6E770E0D6E0D2EFED70C2EFCD719
:1054E6000B2EFAD78D0E0101466F000E476F7AEC30
:1054F60024F0290E0B6E960E0C6E7F0E0D6E0D2E81
:0E550600FED70C2EFCD70B2EFAD78BD6FFD774
:1058220010EE19F00F0E006E010E016EC80EF66E2C
:0E583200570EF76E000EF86ED2EC25F0120045
:10551400200D0A526563686572636865206465736B
:10552400206465766963657320636F6E6E6563746A
:10553400E97320737572206C65206275732049329B
:10554400433120524333203D53434C205243343D96
:065554005344410D0A0062
:10555A002031384632366B32325F4C43443478322B
:10556A00305F4C4344327831365F445331333037FD
:10557A005F55415254315F4932435F323032332EE4
:09558A006D63707069200D0A00C8
:10559300204C69737465206465732061647265735C
:1055A3007365732064652062617365206465766941
:1055B30063657320493243206465636F7576657252
:0855C300746573203A0D0A0023
:1055CB000000007FCDCC4C7B0AD723786F1203757C
:1055DB0017B75171ACC5276EBD37066B95BF5667B4
:1055EB0077CC2B645F700961FFE65B5D08E53C3CA3
:0455FB006042221BCD
:1055FF000000007F000020820000488500007A88AC
:10560F0000401C8C0050438F002474928096189693
:10561F0020BC3E99286B6E9CF90215A0EC782DC129
:04562F00CAF249E290
:105633005F31384632366B32325F4C434434783212
:10564300305F4C4344327831365F44533133303723
:105653005F55415254315F4932435F323032332E0A
:04566300630A0D00C9
:1056670001000000080000004000000000020000E8
:10567700001000000080000000000400000020006F
:1056870000000001000000080000004000000000CA
:10569700010000000A00000064000000E8030000A9
:1056A70010270000A086010040420F008096980056
:0856B70000E1F50500CA9A3B71
:1056BF002056657273696F6E204C434420327831E7
:1056CF0036202B20504346383735342065787465A3
:0656DF00726E650D0A0069
:1056E5000100000010000000000100000010000093
:1056F5000000010000001000000000010000001083
:10570500204465766963652023202066696E6420E0
:09571500617420402020202000D6
:10571E00525443202C32344C43323536206F707441
:05572E00696F6E7300BD
:1057330031384632364B32322036344D487A204D9A
:05574300696B724300D8
:105748002020202020202020202020202020202051
:055758002020202000CC
:10575D00204465766963652023202020403D20206C
:05576D002020202000B7
:1057720020204D6973652061206C2748657572652C
:02578200200005
:105784002050726573656E746174696F6E203A0D92
:025794000A0009
:105796003031323334353637383941424344454661
:0157A6000002
:1057A7003031323334353637383961626364656690
:0157B70000F1
:1057B800303132333435363738394142434445463F
:0457C80000000000DD
:0457CC0000000000D9
:0757D000286E756C6C2900C6
:0C57D7004541303D2535642050747300BE
:0C57E3004541313D2535642050747300B1
:0B57EF00206E6F7420666F756E640002
:0A57FA0044657669636520402000D5
:0758040020736F697420009E
:06580B00444154453A003F
:0658110054494D453A0028
:05581700203D3E2000D1
:05581C00203D3E2000CC
:020000040030CA
:0D000100281F3CFFBF81FF0FC00FE00F4024
:0200000400F00A
:1000000031384632364B32322054657374204932CF
:1000100043204C43442034783230206361720D0019
:1000200055415254203131352C3220382C4E2C3150
:10003000426C7565546F6F746820484330360D000C
:100040005254432044533133303720656E204932B7
:1000500043202020466F73633D31364D487A0D00B2
:100060007265762032392D30332D323032332020F4
:100070004D696B726F4320202056372E36300D00AD
:10008000496E6974204932432062757320343030E0
:100090004B487A2000496E697420525443204453DF
:1000A00031333037202020202000496E69742041F0
:1000B000444320302D3556205241302D3100FFFF72
:1000C000FFFFFFFFFFFFFFFFFFFFFFFFFFFFFFFF40
:1000D000FFFFFFFFFFFFFFFFFFFFFFFFFFFFFFFF30
:1000E000FFFFFFFFFFFFFFFFFFFFFFFFFFFFFFFF20
:1000F000FFFFFFFFFFFFFFFFFFFFFFFFFFFFFFFF10
:00000001FF
